:017FF800D6B2
:017FF900EF98
:030000000200807B
:0300430002011E99
:03004B000200FFB1
:1C00800075810075BE017584FF7800A57A03005AA57A03005BA57A030043A57A4D
:1C009C00030042A57A030055A57A030056A57A030057A57A030058A57E040000FA
:1C00B800A57D1075F100000075E13F43A203A5A9D1B1A5A9D5D3A5A9D0B1D2AF01
:1C00D400759000A5A9C5870200DE000000A57E07005AA50B04A57A07005AA5BE76
:1C00F000047FFF4005D2900200DEC2900200DEC0E0C0F0C0F130C10675F1001249
:1C010C00012530C00675F100120377D0F1D0F0D0E032A5A9C6D3B2933253C0FDF8
:1C01280002012BE5E230E60CE5F554C06000120186020185E543B40211A5A9D424
:1C014400E4A5A9D7F47400F543F542020185B40130A5CA08744C2554F8E5E625BA
:1C01600054F554E5E66009A6E308D5E0FAA5DA08A5A9D4E4E554B54B0CA5CAEB46
:1C017C001201DDA5DAEB02018522E5E6C2D79408702DA5A9C4E285E34485E34579
:1C01980085E34785E34685E34985E34885E34B85E34AA5CAEBA5A9D4E4A5A9C6B4
:1C01B400E21201BCA5DAEB22755800755900E54420E710754301754202E54A4531
:1C01D0004B600A75540022754302754201E54420E64220E53F20E70302020953E2
:1C01EC00E01FB40003020225B40103020376B402030202AEB40303020376020241
:1C0208002453E01FB40003020354B40103020376B402030202FCB4030302037633
:1C02240022E545B40667E546B401117555FF755604755701741275F000020268A4
:1C024000B402117555FF755604755713741275F000020268B403467555FF75567C
:1C025C0004755725741375F000020268C0E0C0F0C2D7954BE5F0954A400CD0F0B0
:1C027800D0E0854AF0E54B020286D0F0D0E085F058F5591203A50202ADB408038C
:1C0294000202ADB400130202ADC0F175F10175F31275F601D0F143E1C022E54536
:1C02B000B40027E549540F42F1E54920E70AE5E130E60C74010202CFE5E130E747
:1C02CC0002740153F180F5F375F30075F602C0F175F10175F31375F601D0F1431B
:1C02E800E1C022754A00754B00754302754201A5A9D1E122C0F1E549540F42F1AF
:1C030400E547B40036E545B4011DE549540F700653E13F02034FE54920E706536F
:1C032000E17F02034F53E1BF02034FB40311E54920E70643E18002034F43E14067
:1C033C0002034FC0F175F10175F31475F601D0F143E1C0D0F10203A1E545B4095E
:1C03580003020362B405060203620203A1C0F175F10175F32075F601D0F143E162
:1C037400C0222253C0FE02037DE542B4020C120395754200754300020394B40186
:1C039000031203A522E545B4050685478F0203A02275F60022A5CA08A5CAEB8584
:1C03AC005584855683855782E5584559700578000203F47800E584601774009380
:1C03C800F5F3A308D55907E558601B14F558B808EC0203EEE0F5F3A308D55907F1
:1C03E400E558600614F558B808EE85835685825788F6A5A9D1E1A5DAEBA5DA0820
:020400002212C6
:0104020001F8
:020403000001F6
:0104050004F2
:0104060001F4
:0104070000F4
:0104080008EB
:020409008680EB
:02040B00495650
:02040D000001EC
:01040F0000EC
:0104100000EB
:0104110000EA
:0104120001E8
:0104130009DF
:0104140002E5
:0104150012D4
:0104160000E5
:0104170001E3
:0104180002E1
:0104190000E2
:01041A0040A1
:01041B0019C7
:01041C0009D6
:01041D0004DA
:01041E0000DD
:01041F0000DC
:0104200001DA
:0104210000DA
:0104220000D9
:0104230000D8
:0104240000D7
:0104250013C3
:0104260003D2
:110427005553422054657374204669726D77617265BD
:00000001FF
